:03F0000002F00813
:03F0610002F003B7
:05F0030012F15380FE34
:03F0640053BEFB9D
:08F06700E5BE30E6FB53C6B81C
:0EF06F00E5C620E6FB43BE0490DF07740AF0FE
:0EF07D0090DF08E4F090DF0C7486F090DF0D59
:0EF08B007483F090DF0E7430F090DF0F74226B
:0DF09900F090DF1074F8F090DF06E4F090C6
:0EF0A600DF11F090DF1A7456F090DF1B74102B
:0EF0B400F090DF147414F090DF157416F090D5
:0EF0C200DF16746CF090DF177403F090DF1807
:0EF0D0007440F090DF197491F090DF1C74E929
:0DF0DE00F090DF1D742AF090DF1EE4F0902A
:0EF0EB00DF1F741FF090DF237488F090DF2485
:0EF0F9007431F090DF257409F090DF2E74FF63
:0EF10700F090DF037404F090DF047422F090A7
:0EF11500DF05E4F090DF0274FFF090DF00747D
:09F12300AAF090DF0174AAF022A9
:04F12C00AA82AB8385
:05F130001ABAFF011BEB
:0EF13500C3E49A74808BF063F08095F0500F65
:04F143007CB07D041B
:05F147001CBCFF011DCE
:06F14C00EC4D70F780DEBF
:01F15200229A
:0DF1530090FE00E0FAC2A8C00212F0649025
:0AF16000000A12F12CD00275E10242
:0EF16A0090DF3BE0FBBB0DF87B00900064C023
:0AF1780002C00312F12CD003D002F4
:08F18200C3EB9A400302F1A562
:0EF18A00900001C00212F12CD00290DF3AE09A
:0DF19800FC74806CFB90FE00F0A502F1827B
:06F1A50075E10475E103B1
:0CF1AB0090DF3BE0FA53021FBA13F5A5F9
:02F1B70080FED8
:06F03700E478FFF6D8FDAD
:08F015007900E94400601B7A58
:05F01D000090F1BD7838
:03F02200007593E3
:0AF0250000E493F2A308B80002050E
:08F02F0093D9F4DAF27593FFA6
:08F03D007800E84400600A7944
:03F04500007593C0
:06F0480000E4F309D8FC0E
:08F04E007800E84400600C7931
:0BF0560000900000E4F0A3D8FCD9FA01
:03F0080075810708
:0AF00B0012F1B9E582600302F00380
:04F1B9007582002239
:00000001FF
